:020000040000FA
:08000000FF308A00DF2E6300CF
:103800000000000000000000FF3E031C0800042C24
:10381000FF3E03190800082CF63E03180C2C080084
:10382000112412240030A000FF300024FF300024B7
:10383000FF300024E3300024A00B142C0800A1006A
:103840001024A10B202C0800220885000800230862
:103850008600080024088700080025088800080062
:103860002608890008002615302C2611302C2B152F
:103870002B0883168900831208002B112B0883164E
:10388000890083120800FF30A700FF30A800FF3036
:10389000A900FF30AA000F30AB0083168900831205
:1038A0000800C2005424C20E420E0F39F63E03181F
:1038B000073E3A3EB62608000330B7000F30B80086
:1038C0000F30B9000F30BA0008000030B7000030E8
:1038D000B8000F30B9000F30BA00080033083B06BB
:1038E000B306BB0634083C06B406BC0635083D06E4
:1038F000B506BD0636083E06B606BE0608002F0809
:103900003106AF06B1062E083006AE06B006080036
:1039100033083B0637053F30031DAD0034083C0635
:1039200038053F30031DAD0035083D0639053F30F1
:10393000031DAD0036083E063A053F30031DAD00BD
:1039400008002E08831203178D00831203132F081B
:10395000831203178F0083120313080083120317C7
:103960000E0E831203130F39B300831203170E08D0
:10397000831203130F39B400831203170C0E831242
:1039800003130F39B500831203170C0883120313B6
:103990000F39B600080083120313330E3404831268
:1039A00003178E0083120313350E36048312031798
:1039B0008C00831203130800831603178C170C1452
:1039C00000000000831203130800831603178C17EE
:1039D0000C158B1355308D00AA308D008C1400000F
:1039E00000000C11831203130800831603178C13B5
:1039F0000C14831203178E0183120313080083161D
:103A000003178C130C158B1355308D00AA308D00C5
:103A10008C148C18092D0C1183120313080041100B
:103A20000800AE0A0319AF0A08003208F63E031870
:103A3000073E3A3EAD00080008000030B3000230F7
:103A4000B4000030B5000130B60008002030B300EB
:103A50001530B4002D30B5003B30B6000800000032
:103A600000000000000000303306031D0800003095
:103A70003406031D080000303506031D0800003021
:103A80003606031D080041140800831203172F3067
:103A90008D001D308F0083120313DC243308831242
:103AA00003178D0A03198F0A0C0683120313031DD3
:103AB0000800DC243408831203178D0A03198F0AC7
:103AC0000C0683120313031D0800DC24350883123F
:103AD00003178D0A03198F0A0C0683120313031DA3
:103AE0000800DC243608831203178D0A03198F0A95
:103AF0000C0683120313031D080041140800411033
:103B0000332545250800831203172F308D001D3003
:103B10008F00831203133308831203178C000319D9
:103B20008F0A83120313E5243408831203178C00D1
:103B300003198F0A83120313E52435088312031730
:103B40008C0003198F0A83120313E52436088312AD
:103B500003178C0003198F0A83120313E52408004E
:103B6000831203172F308D001D308F008312031333
:103B7000DC24831203178D0A03198F0A0C088312A1
:103B80000313B300DC24831203178D0A03198F0A71
:103B90000C0883120313B400DC24831203178D0A6C
:103BA00003198F0A0C0883120313B500DC24831257
:103BB00003178D0A03198F0A0C0883120313B6002A
:103BC00008002D08B626122406301324831603138A
:103BD00000309F008312031300308A0000000000B1
:103BE00000000328831203170F081B3C83120313E2
:103BF000031CC110080083120317EE308D001D3026
:103C00008F0083120313080083120317EF308D0017
:103C10001D308F0083120313080083120317F03046
:103C20008D001D308F0083120313080083120317C9
:103C30000F0883120313031D0800831203170D08D6
:103C400083120313003E0319FB2DFF3E0319042EBC
:103C5000FF3E03190D2E0800F225162683120313CA
:103C60000800A009723F83120313C11083120317C7
:103C70000D0883120313063C031D472E83120317FE
:103C800031308D001E308F00831203130800831221
:103C9000031732308D001E308F008312031308008B
:103CA00008005C240130AC00080065240230AC0040
:103CB00008005C240330AC0008000800AF01AE012E
:103CC00036080C3C0319512636080D3C03195526BD
:103CD00036080F3C0319592636080E3C03195D2699
:103CE00008005026F52408002C26DC240800332682
:103CF000DC240800A1242C08023C031971262C089E
:103D0000013C031974262C08033C03197726AE24C2
:103D10000800502683120313C118FF2408002C2624
:103D2000C118E52408003326C118E5240800A124A1
:103D3000CB24C1142C08023C031989262C08013C11
:103D400003198F262C08033C031993266E247A2628
:103D5000882408006E247A2688242D083F3A031D03
:103D600008004C30AD006E2497260800C0003524B2
:103D70003D244008C3000A30C40033242F300224FD
:103D800043183524431C3324C30CC317C40BBE2E65
:103D9000372408000310091DDC2EC6013130C50090
:103DA000091DFF3EC50BD02ECE3E193EC60C031C8E
:103DB0000319DB2ECE2E4609031CCA2E08008316DB
:103DC000031307309F00831203130919E62D4324C0
:103DD0004114CA267F39AD009F3E0318AD12323020
:103DE00000244118F82E2D08483C03197F25342F54
:103DF0002D08473C0319E1252D08483C03197F2570
:103E00002D08493C031911252D084C3C0319AA26FD
:103E10002D08503C0319E1252D08513C0319B0250C
:103E20002D08523C03197A262D08533C03190F25FF
:103E30002D08543C031926252D08553C03198325CC
:103E40002D08563C03191D252D08573C03199726AC
:103E50002D08583C03195E262D085A3C03191C25D1
:103E60002D084E3C031915253308B2003408B30061
:103E70003508B4003608B5002D08BF3E0318F93EDA
:0C3E8000113EB6002D084118B626E92EB0
:02400E00723FFF
:00000001FF
